:10000000051A0428A9018D01061D0428802306195C
:10001000062886190C2804288316F83085000C3031
:100020008600843081008312850186018B0188302F
:100030008400AA01A601A701AF012B20061D2428D8
:10004000A61FA60A49211E282B2006191D28A61F17
:10005000A60A49212528A70A26080319832864002F
:10006000A6010D10FD3E031C0D140318A701E73077
:100070002A070318AA012A088207B228C428D5280B
:10008000E628F528E628F528E628F528E628F528C4
:10009000E628F528E628F528E628F528E628FE28AB
:1000A0000A2919292B2937294329AA010D1C122AAB
:1000B0000C080319C12916081706180619061A068E
:1000C000031D7A298C19152AA701AD018D11170876
:1000D000E0390319802A203A0319CD2AC03A0319BE
:1000E000102B603A0319F82AC039C03A0319272B9C
:1000F00008000D1908008D1C0800180897008D10C5
:10010000E039E03A7128AA01A701082A8E0A0E08F0
:100110000739820767298A29AE296729CC29E0296E
:100120006729F429170898000730160582075E2A08
:100130005E2A5E2A5E2A5B2A6D2A08000800240EC9
:100140000F3982070F340734073403340334013482
:1001500001340034003401340134033403340734EF
:1001600007340F34EC302707031CC129AA0A980171
:1001700099018C019B018901001408088F00890AEC
:1001800000140808900008000D1CAA0A023089001B
:10019000001408089100FE3E031C91090A308900F2
:1001A00000140808950000000800AA0A0D18AA010A
:1001B0000530890000140808E83E0318FF30203E8F
:1001C0009200890A0014080893000800AA0A031084
:1001D0000D1803149A0D09308900001408089400C2
:1001E0008D127F39031D8D16A029AA0A0D1CFB282C
:1001F0001A1CAA0136291A18AA01142A0D1C03294F
:100200001A1CAA0906291A18AA0900009B0A1B0829
:10021000AA079B290230AA001A0896000D18AA0105
:10022000961BAA01160803198C14903E03188C150E
:10023000A0290230AA001A0897000D18AA01160872
:100240000F0603190C148D1E842914087F39160615
:1002500003198C1608000D1832290230AA001A085A
:100260009800142A1830AA008D100D11032A0D18B9
:100270003E290230AA001A089900142A1830AA0050
:100280008D140D11032AAA0A0D1CAA018D140D1537
:10029000362912080102031C86280430A807120818
:1002A0008102A307031C0B2AAE0AA40A0319AD0A94
:1002B0002408C03903389C000D1E9C150D1A1C160D
:1002C0001C1F9C169F202405031D1C150800FB30D5
:1002D0002E0703188D11130803197F292D02031807
:1002E000A90129082802031885290D1E8029061056
:1002F000861405152408783903199C100800712903
:10030000861006140515A0299F2905112F088604BB
:1003100000009F2911308900001408081D050319E9
:10032000AA291D18A82916308900001408081C05E0
:10033000031DAC2906162408063903191C100000F9
:1003400008002408063903191C10000000000800EA
:10035000061636290612C1290612F4281230890021
:10036000001408081D050319C8291D18C0291730D5
:100370008900001408081C05031DCA298616842953
:100380008616151FC6290330AF009B29AF019B2994
:100390008612C1298612F428133089000014080837
:1003A0001D050319DC2918308900001408081C05F4
:1003B000031DDE2906179B290613C12906137A2976
:1003C00014308900001408081D050319F02919309C
:1003D0008900001408081C05031DF22905149B2937
:1003E0000510C12905107A29153089000014080864
:1003F0001D050319042A1A308900001408081C0579
:10040000031D062A85149B298510C12985107A2988
:10041000092A0A2A0C2A0D2A0E2A0F2A102A5728DE
:10042000112A052A132AFD28072A0D1D8D1D0800F3
:10043000A701AE0142220038031908008D1C922842
:100440001608743A0319772A083A031D0800180899
:1004500088001708063A03190800013A0319080032
:100460001B3A031D362A5130880588141708A0232B
:100470008A0189003F3A03190800640083160815B1
:100480008523BA2A16081E06031D522A17081F06BE
:10049000031D522A18082006031D522A1908210696
:1004A0000319FF3416089E0017089F001808A000C3
:1004B0001908A10000341C3097006A2A2503970010
:1004C0000310970D03180800970D03180800033058
:1004D00016059707961D772A272A961D722A18084F
:1004E000A500080025081806031D0800BA2A1708E9
:1004F000A0238A0189008F231806031D0800BA2A49
:100500000D19080017088D188E2A0319A42A013A1C
:100510000319AB2A0E3A0319BA2A0800123AFE3917
:10052000031D08004222003803190800981B080028
:10053000180803199D2A1718803888000930890087
:1005400083160815852308009D01A9018C1C08004D
:100550008D15AE017928A9019D0109308900880116
:100560008316081585230A30890002308800831617
:1005700008158523640006148610051506168616D0
:1005800081010530AC00011FC32A0113AC0BC32A43
:10059000051106128612AE0108008D1C08003F30BE
:1005A0001706031D08000123003A0319EE2A103034
:1005B000981F8D067F3098050319F42A98030319B4
:1005C000F42A18039E0010081102031C03019F0067
:1005D0006C23A10D200D1007A900A2000D1D08001D
:1005E0000D111908980079280030A900A200EE2A00
:1005F0000D1908000C18FE2A8C1A792817089D007E
:10060000792810308D1A082B0D1215188D06FF341D
:100610008C18042B8C1E00340D12941B8D06052B98
:100620008C1C0C18142B08000D1D080017089600D0
:10063000F739E43A031D0800422200380319080084
:100640001808970019089800961D772A272A0D196F
:1006500008000123003A031979281030971E8D06EF
:10066000AB0197309E0010081102031C3B2B9F002A
:100670006C2320089F0049210310171A0314170D3B
:100680001F399E00FC309E07031C542B151A592B52
:100690006C23A10DA00DA10DA00DA10DA00DA10D0C
:1006A000200D1007A9005E2BA9019E1C5E2BA20144
:1006B0006A2B1B301E0789008F23A90029082206F8
:1006C00003196A2B2908A207220CAC002908A200F2
:1006D0002C08A90029087928A001A101AC01083043
:1006E0008E009E0C031C7A2B2C08A0071F08A10764
:1006F0000318A00A03109F0DAC0D8E0B712B080080
:100700000E308E008E0B822B080055308900AA30E7
:100710008900881488188A2B081183120800001495
:0407200008080800BD
:10074000AC00E33E031CAC2BBF3E03183F342E3EEF
:10075000031C3F34ED30AC0703308A002C088207BD
:10076000003401343F343F3402343F340334043422
:1007700005343F3406343F343F343F343F343F3454
:100780000734083409343F343F343F343F343F3476
:100790003F343F343F343F340A340B340C340D348F
:1007A0000E340F341034113412341334143415341D
:1007B00016341734183419341A343F343F341B3488
:1007C0001C341D341E341F3420342134223423348D
:1007D0002434253426342734283429342A342B343D
:1007E0002C342D342E342F343034313432343334ED
:0607F000343435343634C8
:02400E00FE3F73
:1042000003000100000066000D0007000000000030
:10421000000000000200000000000000000000009C
:104220000000100001000200040010000000000067
:10423000000000008000010006000C0010001400C7
:1042400018001C00200024002A00300036003C002A
:1042500044004C0054005C00660070007C00880044
:0E4260009800A800BC00D000E600FC00FF00A3
:00000001FF
